:020000021000EC
:10E000004BC0000066C0000064C0000062C0000099
:10E0100060C000005EC000005CC000005AC000008C
:10E0200058C0000056C00000EFC3000052C00000FE
:10E0300050C000004EC000004CC000004AC00000AC
:10E0400048C0000046C0000044C0000042C00000BC
:10E05000EBC100003EC000003CC000003AC0000020
:10E0600038C0000036C0000034C0000032C00000DC
:10E0700030C000002EC000002CC000002AC00000EC
:10E0800028C0000026C0000024C0000022C00000FC
:10E0900020C000001EC0000011241FBECFEFD0E240
:10E0A000DEBFCDBF11E0A0E0B1E0EEE2FEEE01E0A8
:10E0B0000BBF02C007900D92A63DB107D9F721E032
:10E0C000A6EDB1E001C01D92A43FB207E1F731D047
:10E0D000ACC696CF8091D601882351F18091E6019C
:10E0E0009091E701A091E801B091E9018827409162
:10E0F000DE015091DF016091E0017091E10148176C
:10E1000059076A077B07A1F025E0FA0160935B00DD
:10E1100020935700E89507B600FCFDCF8093DE0101
:10E120009093DF01A093E001B093E1011092D6013A
:10E13000089584B7877F84BF88E10FB6F8948093F1
:10E140006000109260000FBE90E080E80FB6F89477
:10E1500080936100909361000FBEC1E0C5BF82E073
:10E1600085BF37D3C0936F0083E08093810078949C
:10E1700011E043E0E42E01E054E0D52E66E0C62E27
:10E1800073E0B72EE2E0AE2E80910001882309F4FF
:10E1900034C181E091E097D5F82E882309F428C195
:10E1A000C0E0D0E0FC1609F423C181E091E0ABD5DA
:10E1B0009091D701992311F08A33D1F41092DD01A7
:10E1C0004090E2015090E3016090E4017090E5011D
:10E1D0004092E6015092E7016092E8017092E901F5
:10E1E0001092DA018A3309F001C10093D701FEC011
:10E1F0002FEB280F263010F4875304C080538A3049
:10E2000008F0F4C02091D90140E1249F900111242D
:10E21000282B2093D9018091DA0181278093DA019C
:10E220008111E4C08091DD01963009F4CEC0820FE7
:10E230008093DD01933059F100F5913019F192305E
:10E2400009F0D2C0422F50E0542F44278091E601BC
:10E250009091E701A091E801B091E901840F951F29
:10E26000A11DB11D8093E6019093E701A093E80101
:10E27000B093E901B092D701B9C09430F9F095306C
:10E2800049F1B2C02093DC01A092D701AFC0409009
:10E29000E6015090E7016090E8017090E901420EBC
:10E2A000511C611C711C4092E6015092E701609282
:10E2B000E8017092E901D092D70198C02093DB0168
:10E2C0008091DC01882311F085E001C086E0809315
:10E2D000D7018CC08091DC0181508093DC0140909B
:10E2E000E6015090E7016090E8017090E901411467
:10E2F00090EE590691E06906710428F01092D7015A
:10E300001092D60173C080FF03C02093D8016EC065
:10E31000422F50E0542F44278091D801482B809100
:10E32000DB01823009F433C0843009F43AC0811132
:10E3300045C08091D601811113C08091DE0190917A
:10E34000DF01A091E001B091E101FC01A0935B002D
:10E35000E0925700E89507B600FCFDCF0093D60188
:10E360000A01F20160925B0010935700E8951124B6
:10E3700042E0440E511C611C711C4092E601509217
:10E38000E7016092E8017092E901A4DE17C060E045
:10E3900070E094E0440F551F661F771F9A95D1F7E0
:10E3A00005C060E070E0BA01552744274093E201C0
:10E3B0005093E3016093E4017093E5018091DC01E7
:10E3C000811114C0C092D70111C0422F50E0819535
:10E3D00090E04817590751F47DDE8091DB018130D0
:10E3E00029F41092000102C01092D7012196DACED2
:10E3F00081E091E01BD4C2D3C7CE8091E000816060
:10E400008093E00082E49CED9093F5018093F40109
:10E410002CE088E190E00FB6F894A8958093600016
:10E420000FBE20936000FFCF1F920F920FB60F9286
:10E4300011240F900FBE0F901F9018950895089506
:10E4400081E091E0B6D31092D701089581E091E088
:10E4500083C4292F33272230310559F02330310569
:10E4600069F021303105D9F482E190E029E831E00A
:10E470001AC080E290E029E631E015C09927833088
:10E48000910568F4FC01EE0FFF1FED5EFE4F208149
:10E490003181FC01E05FFE4F808190E004C080E0AC
:10E4A00090E020E030E0FA0131832083089507B640
:10E4B00000FCFDCFF999FECF23E0FB0180935B00C8
:10E4C00020935700E89507B600FCFDCF81E18093CB
:10E4D0005700E895089507B600FCFDCFF999FECFE7
:10E4E00025E0FB0180935B0020935700E89507B679
:10E4F00000FCFDCF81E180935700E895089507B6B1
:10E5000000FCFDCFF999FECF21E00A01FB018093C9
:10E510005B0020935700E8951124089521E2FC0147
:10E52000209357008491089529E0FC01209357001F
:10E5300084910895E1E0F0E089E0809357008491B0
:10E54000089507B600FCFDCFF999FECF809599E0BC
:10E55000E1E0F0E0082E90935700E89508952091AF
:10E56000F2013091F3012617370748F06115710564
:10E5700039F42091E8002E772093E80001C0B9011A
:10E58000FC0120E06115710591F18EB38823E1F162
:10E590008530E1F18091E80083FD3AC08091E80088
:10E5A00082FF06C08091E80082FF24C080E00895C9
:10E5B0008091E80080FFE6CF8091F2009091F30017
:10E5C0006115710551F08830910538F4219120933F
:10E5D000F100615071090196F3CF21E0089709F02D
:10E5E00020E08091E8008E778093E800CBCF211166
:10E5F000CCCFD8CF8EB3882339F0853039F08091D5
:10E60000E80083FFCFCF04C082E0089583E008953F
:10E6100081E008958F708093E900EBEEF0E0808157
:10E6200081608083EDEEF0E010826093EC00408327
:10E630008091EE00881F8827881F08950F931F93ED
:10E64000CF93DF93062FEC0110E0101771F1988142
:10E65000992341F12C81E981FA817B81892F8F7087
:10E66000873010F080E022C0223010F056E001C068
:10E6700052E028E030E040E02E173F0720F44F5FE3
:10E68000220F331FF9CF4295407F452B692F661F1C
:10E690006627661F90E4799F90011124622BBADFF0
:10E6A000882301F31F5F2596D0CF81E0DF91CF91C2
:10E6B0001F910F9108958091EC0187FD05C0809115
:10E6C000E80080FF0DC010C08091E80082FD04C00A
:10E6D0008EB38111F9CF08958091E8008B7707C040
:10E6E0008EB38111ECCF08958091E8008E778093EE
:10E6F000E80008958091E4009091E50045E62091BE
:10E70000EC0020FF20C02091E80020FD20C02EB3A7
:10E71000222389F0253089F02091EB0025FD0FC0E0
:10E720002091E4003091E5002817390741F341506A
:10E7300041F0C901E4CF82E0089583E0089581E0CB
:10E74000089584E008952091E80022FFE0CF80E062
:10E7500008950F931F93CF93DF9349D050D0C8ED06
:10E76000D0E088818F7788838881806888838881DA
:10E770008F7D8883E7EDF0E080818068808319BC1D
:10E780001EBA1092EA0100EE10E0F80180818B7F42
:10E79000808388818160888342E060E080E03ADFA6
:10E7A000E1EEF0E080818E7F8083E2EEF0E0808118
:10E7B00081608083808188608083F80180818E7F82
:10E7C0008083888180618883DF91CF911F910F9131
:10E7D0000895E8EDF0E080818F7E8083E7EDF0E042
:10E7E00080818160808381E08093EB01B2CFE8ED8E
:10E7F000F0E080818C7F80831092E2000895109277
:10E80000DA001092E10008951F920F920FB60F9256
:10E8100011240BB60F922F933F934F935F936F93F7
:10E820007F938F939F93AF93BF93EF93FF938091C9
:10E83000DA0080FF1BC08091D80080FF17C0809154
:10E84000DA008E7F8093DA008091D90080FF0BC0C0
:10E850008CE089BD8EE089BD09B400FEFDCF81E06A
:10E860008EBBECDD03C019BC1EBAE9DD8091E1006E
:10E8700080FF17C08091E20080FF13C08091E2000A
:10E880008E7F8093E2008091E20080618093E200BD
:10E890008091D80080628093D80019BC85E08EBB3F
:10E8A0006CD18091E10084FF2EC08091E20084FF52
:10E8B0002AC08CE089BD8EE089BD09B400FEFDCF81
:10E8C0008091D8008F7D8093D8008091E1008F7E69
:10E8D0008093E1008091E2008F7E8093E20080913E
:10E8E000E20081608093E2008091EA01882311F0C8
:10E8F00084E007C08091E30087FF02C083E001C08D
:10E9000081E08EBB3AD18091E10083FF21C08091EC
:10E91000E20083FF1DC08091E100877F8093E100CA
:10E9200082E08EBB1092EA018091E1008E7F80939D
:10E93000E1008091E2008E7F8093E2008091E2000E
:10E9400080618093E20042E060E080E063DE15D108
:10E95000FF91EF91BF91AF919F918F917F916F91B7
:10E960005F914F913F912F910F900BBE0F900FBE73
:10E970000F901F9018951F93CF93DF9300D0CDB7C2
:10E98000DEB7ECEEF1E08091F100819381E0E43FAD
:10E99000F807C9F75BDD8091E80083FFDAC090914A
:10E9A000EC018091ED01853009F465C030F48130CF
:10E9B00059F168F0833041F1CCC0883009F49CC033
:10E9C000893009F4ABC0863009F0C3C075C09038F7
:10E9D00081F0923809F0BDC08091F0018F70809372
:10E9E000E9009091EB0095FB992790F91092E900CE
:10E9F00001C090E08091E800877F8093E8009093C9
:10EA0000F1001092F10083C0292F2D7F09F0A1C0E1
:10EA1000923009F09EC09091EE01911126C0209194
:10EA2000F0012F7009F495C02093E9009091EB005C
:10EA300090FF1BC0833021F48091EB00806213C0F3
:10EA40008091EB0080618093EB0081E090E0022EEA
:10EA500001C0880F0A94EAF78093EA001092EA0056
:10EA60008091EB0088608093EB001092E900809128
:10EA7000E800877F4FC091116CC01091EE011F77A5
:10EA80008091E3008078812B8093E3008091E800FF
:10EA9000877F8093E8000FDE8091E80080FFFCCF45
:10EAA0008091E30080688093E300112311F083E0FC
:10EAB00001C082E08EBB4DC09058923008F049C032
:10EAC000AE014F5F5F4F6091F0018091EE01909138
:10EAD000EF01BFDC009709F43CC02091E800277FDC
:10EAE0002093E800BC0189819A8139DD8091E8009A
:10EAF0008B778093E8002DC0903859F58091E8001D
:10EB0000877F8093E8008091EA018093F1008091F3
:10EB1000E8008E778093E800CEDD1BC0911119C00C
:10EB20009091EE019230A8F48091E800877F809365
:10EB3000E8009093EA01BFDD8091EA01811104C0F1
:10EB40008091E30087FF02C084E001C081E08EBBBA
:10EB500077DC8091E80083FF0AC08091E800877F1E
:10EB60008093E8008091EB0080628093EB000F902F
:10EB70000F90DF91CF911F9108950895CF938EB399
:10EB80008823A9F08091E9008F709091EC0090FFAC
:10EB900002C090E801C090E0C92FC82B1092E90094
:10EBA0008091E80083FDE7DECF70C093E900CF914C
:10EBB0000895CF93DF93EC011E861D8688E18D8733
:10EBC00082E08C83898761E0CE01019637DD88235E
:10EBD00031F061E0CE010696DF91CF912FCD80E03C
:10EBE000DF91CF9108952EB32430F1F4FC0181819F
:10EBF0008F708093E9008091F2009091F300892B4F
:10EC000089F09091E8008091E8008E778093E80089
:10EC100095FD08C06FDD811108C08091E8008E77F6
:10EC20008093E80080E0089582E00895CF93DF9319
:10EC3000EC018EB3843009F043C089818F708093DA
:10EC4000E9008091E80080FF02C0CE01CCDF8E8514
:10EC50008823B1F12E812F7081E090E0AC0102C0D9
:10EC6000440F551F2A95E2F74093EA001092EA00FC
:10EC700029812F70022E01C0880F0A94EAF7809331
:10EC8000EA001092EA008E818F708093E9008091F3
:10EC9000EB0080618093EB008091EB0088608093B3
:10ECA000EB0089818F708093E9008091EB00806197
:10ECB0008093EB008091EB0088608093EB001E86D0
:10ECC000DF91CF9108952EB3243019F080E090E0C9
:10ECD0000895FC0186818F708093E9008091E8009F
:10ECE00082FFF4CF8091F2009091F300009731F40D
:10ECF0002091E8002B772093E80008958091F2009E
:10ED00009091F30008952EB3243019F08FEF9FEF08
:10ED10000895FC0186818F708093E9008091E8005E
:10ED200082FFF4CF8091F2009091F300892B21F0C3
:10ED30002091F10030E002C02FEF3FEF8091F20010
:10ED40009091F300892B29F48091E8008B778093D0
:10ED5000E800C90108950895CF93DF93EC018091F5
:10ED6000E80083FF5FC0888190E02091F00130913E
:10ED7000F1012817390709F055C08091ED01813064
:10ED800051F120F0823009F43DC04CC08091EC017B
:10ED9000813A09F047C08091E800877F8093E800BE
:10EDA0008091E80080FD04C08EB38111F9CF3AC094
:10EDB000EB85FC85DF010D900020E9F7BD01615076
:10EDC00071096E1B7F0B7093F1006093F1008B85CE
:10EDD0009C85C5DB14C08091EC01813A19F58091C6
:10EDE000E800877F8093E8008091E80080FD04C000
:10EDF0008EB38111F9CF16C08D858093F100DF911C
:10EE0000CF9159CC8091EC01813261F48091E8007E
:10EE1000877F8093E8004FDC81E08E87CE01DF9111
:0EEE2000CF9199CFDF91CF910895F894FFCF55
:10EE2E000100834000000104400000019B0100002E
:10EE3E0004183065014B01190130034C0055004692
:10EE4E0000410020005000720069006E00740065E1
:10EE5E00007200200042006F006F0074006C006FA3
:10EE6E000061006400650072000000180344006534
:10EE7E000061006E002000430061006D00650072AD
:10EE8E0000610000000403090409022000010100D2
:10EE9E0080320904000002070102000705830240C8
:10EEAE0000050705040240000512011001000000D4
:10EEBE0008EB036B200100010200014D46473A4763
:10EECE00656E657269633B4D444C3A47656E65727B
:10EEDE0069635F2F5F546578745F4F6E6C793B4347
:10EEEE004D443A313238342E343B434C533A50521F
:06EEFE00494E544552008C
:10FFA0000C9457F20C946BF20C947FF20C948EF23A
:10FFB0000C9494F20C949AF20C94A1F20895089582
:06FFC00008950895089564
:10FFE000DFCFE0CFE1CFE2CFE3CFE4CFE5CFE6CF85
:08FFF000E6CFE6CFE6CFE6CF35
:08FFF80000E0010020DFFBDC4A
:040000031000E00009
:00000001FF
